:10000000830100308A00042883168130990024304F
:10001000980083129030980083124420A000503042
:1000200020020319202849302002031923284C30CC
:10003000200203192C2853302002031934280D28DC
:100040004F3048200D28493048202030482030309B
:100050004820103048200D283A200008A3004C30DA
:100060004820230848200D283A204420800053309F
:1000700048200D28442084004420A1002118422853
:1000800083134328831708008C1E44281A0808008D
:080090000C1E4828990008002D
:00000001FF
